:020000040001F9
:18F000004FF0200383F3118872B6024B9D4600F08BBAC046F82C0020B0
:20F018009B4900200860086830B900BF0868401C086008680028F8D0704710B500F05FF8FD
:20F03800022000F0CCFDFFF7EBFF012000F0ACFD0024092C0CDA022000F0C1FDFFF7E0FF5F
:20F05800022000F0A1FDFFF7DBFF641C092CF2DB00F055F8FFF7D4FF10BD38B585480124E4
:20F078000460042000F05EFC042000F0FEFC0128FAD14FF4A06000F0D3FD7F487F490460AE
:20F0980008688008FCD300250A2D05DA284600F07BFD6D1C0A2DF9DB794D204600212A462F
:20F0B80000F0F2FD022000212A4600F0EDFD75480421016002250560204600F065FD2846D7
:20F0D80000F062FDFFF7A9FF6F496FF00042A1F108000260086820F00200086038BD10B532
:20F0F80069480124001D0460022000F04DFDFFF787FF204600F063FDFFF782FF10BD08B512
:20F11800022000F05CFDFFF77BFF012000F057FDFFF776FF022000F037FDFFF771FF01205F
:20F1380000F032FDFFF76CFF08BD70B50646072417D40125022000F042FDFFF761FF05FA1F
:20F1580004F0304203D1284600F039FD02E0284600F01AFD022000F017FDFFF751FF641E84
:20F17800E8D5022000F02BFD012000F00DFDFFF747FF44482030006810F002004FF00001A3
:20F1980000D101210C46022000F0FEFCFFF738FF204670BD2DE9F04180460025072419D4FC
:20F1B800384F0126022000F00AFD304600F0ECFCFFF726FF07F120000068800803D306FA29
:20F1D80004F02843C5B2022000F0DEFCFFF718FF641EE7D5022000F0F2FCFFF711FFB8F15B
:20F1F800000F03D1012000F0CFFC02E0012000F0E6FCFFF705FF022000F0C6FCFFF700FFA0
:20F218002846BDE8F08170B515460E460446FFF766FF6000C0B2FFF788FF0024A54205DD9D
:20F23800A05DFFF782FF641CA542F9DCFFF767FF012070BD70B515460C460646FFF74FFFFA
:20F25800700040F00100C0B2FFF76FFF002604E00120FFF79FFF3055761C681EB042F7DCFE
:20F278000020FFF797FF3055FFF749FF002070BD040100200C4009402820086028200840C0
:20F2980000600044A020024008000840704700F069BA2DE9F04190460F46064617B306F018
:20F2B800FF00C0F58070874204D906F0FF04C4F5807400E03C46002500E06D1C3046214679
:20F2D8004246FFF7E4FF012801D00A2DF5D30A2D02D34FF0FF3006E004EB08008046A619E0
:20F2F8003F1BDCD10120BDE8F08100F062BA2DE9F04190460F46054607B305F0FF00C0F58C
:20F318008070874204D905F0FF04C4F5807400E03C46002600E0761C214628464246FFF74D
:20F33800E4FF012801D00A2EF5D30A2E02D34FF0FF3004E0A04465193F1BDED10120BDE848
:20F35800F08108B501216A46FFF7A3FF9DF8000008BD08B502216A46FFF79BFFBDF80000CE
:20F3780008BD08B504216A46FFF793FF009808BD08B58DF8001001216A46FFF7B6FF08BDA5
:20F3980008B5ADF8001002216A46FFF7B0FF08BD08B5009104216A46FFF7A9FF08BD2DE90A
:20F3B800FF410D180446A5423AD94FF0FF0800273E4600E0761C281B102801D9102100E0C3
:20F3D800291B20466A46FFF764FF012801D00A2EF0D3384607E01DF80010FF2900D00127C3
:20F3F80000F80D80401C291B102901D9102100E0291B8142EFD887B1002600E0761C281BCB
:20F41800102801D8291B00E0102120466A46FFF76CFF012801D00A2EF0D31034A542C6D839
:20F438000090BDE8FF81F0B5ADF1140D0E18FF240546AE4222D9002700E07F1C701B1028B7
:20F4580001D9102100E0711B28466A46FFF721FF012801D00A2FF0D3002104E011F80D00D8
:20F4780020400446491C701B102801D9102000E0701B8842F2D81035AE42DCD8204605B095
:20F49800F0BD0000624B002119601968884206D91A461968491C196011688842F9D87047AC
:20F4B80010B55C4C01210A46204600F0FAFB0121204600F019FC10BD0246880000EBC10034
:20F4D80000F5F8300C2100F099BB0246880000EBC10000F5F8300C2100F099BB7CB50646FF
:20F4F8004D4C002000904D4D05E0204604216A4600F084FB503C0098B0F1FF3F01D0A542C7
:20F51800F3D904F150005021324600F080FB7CBD7FB5054628083BD2082D00D9082500241A
:20F53800A54243D94CF25030FFF7ACFF00F060FB4CF25030FFF7A6FFE1B26846FFF7BCFFBB
:20F55800009820F00040B0F5F83F1DD00198D8B1000819D2684600F0FFF8A8B94CF2503019
:20F57800FFF790FF00F044FB4CF25030FFF78AFF684600F0EEF838B9019840F00040019073
:20F59800E1B26846FFF7A1FF641CA542CAD80DE04CF25030FFF776FF00F02AFB4CF250308A
:20F5B800FFF770FF25F00040FFF798FF4CF25030FFF768FF1A4C216841F0020121602168A4
:20F5D80041F001012160174E00253560FFF75AFF1549086840F00040086014490420086062
:20F5F800206840F002002060206840F001002060356000F088FBFEE7704708B50A4908685C
:20F6180040F0004008600120FFF782FFFEE7C0460001002000400340B0FC0100D0FA01005B
:20F638000800084000000840040009401021084008B500F4F831B1F5F83F02D14FF0FF305C
:20F6580009E0C0F30F30000300F00FFB10B14FF0FF3000E0002008BD08B500F0F7FA10B167
:20F678004FF0FF3000E0002008BDD0B50A4641F221030021082915DAC40B0027E60300D023
:20F6980001273E46400080B232F07F0701D040F001000EB1584080B25200D2B2491CC9B24B
:20F6B8000829E9DBD0BD2DE9F84F8946834600254FF6FF7ADBF8000020F00048DBF8047066
:20F6D800B9F1000F01D0444635E0254C33E0B7F5807F01DC3E4601E04FF48076204A40464F
:20F6F800314600F08BFA40F6FF7010EA080F05D1B9F1000F02D04046FFF79AFFB9F1000F21
:20F7180002D10020164C04E0154841463246FFF7A3FF78B90025AE4208D921785046FFF758
:20F73800A4FF8246641C6D1CAE42F6D80025BF1BB04400E06D1C002F01DD052DC7D3BBF897
:20F758000A00824501D1002001E04FF0FF30BDE8F88F0121FFF7A7BF0021FFF7A4BFC04655
:20F77800000000207CB516460D4604468DF80140200A8DF80000210C0020090400D0012067
:20F79800503069460222FFF73EFD78B1210C0020090400D0012050302A463146FFF74AFDB5
:20F7B80010B14FF0FF3003E0012001E04FF0FF307CBD30B5ADF5827D0C46054611468DF877
:20F7D8000150280A8DF8000022460DF1020000F01EF80020290C090400D001205030A21C0A
:20F7F8006946FFF710FD08B101200EE0290C0020090400D001205030A21C6946FFF703FD41
:20F8180008B1012001E06FF0030041B030BD002A4AD05FEA000C8B071CD1830722D1102A06
:20F8380008D370B4103A78C978C0103AFBD270BC103238D0042A2CD3082A05D30C2A24BF11
:20F8580008C908C008C908C008C908C092072AD0920F22E00B780370491C401C521E22D076
:20F878008B07F7D1C30714D18307D8D0121F12D308C903801B0C4380001D121FF8D20AE0DF
:20F8980008C903701B0A43701B0A83701B0AC370001D121FF4D2121D05D00B780370491C51
:20F8B800401C521EF9D160467047002213460A46194671B510F0030F0BD0002A82BF00F89D
:20F8D800011BB2F1010210F0030FF6D1002A08BF71BD11F0FF0141EA0121042A18D341EAC4
:20F8F8000141082A0FD30E46102A08D30C460D46B2F10F0312F00F0272C0103BFCD812F071
:20F91800080F18BF42C012F0040F18BF40F8041B12F0020F18BF20F8021B12F0010F18BF94
:20F93800017071BD41080BD342F23012C4F20802116841F001011160916D41F0010191656F
:20F95800810807D342F23412C4F20802116841F001011160C10807D342F23812C4F20802F4
:20F97800116841F001011160410907D342F28C12C4F20802116841F001011160800907D31C
:20F9980042F28411C4F20801086840F001000860704700001348B0B5B0F1FF3F01D000F0A7
:20F9B8008DF8114D1148A84210D01148114CA0420CD0001BC71054F8040B10F8011B55F8F7
:20F9D800212054F8041B90477F1EF4D10A4D0B4CA54205D002E054F8040B8047A542FAD10A
:20F9F800B0BDC046FFFFFFFF28FE010034FE010050FE010040FE0100000000000000000098
:20FA18002DE9F041054615F8017B90460E461CE0B8F1000F05F101050BD0FF2C09D80220D0
:20FA380015F8011B401E41EA0424F9D101E0042C02D315F8011B00E0394630462246FFF7C8
:20FA580038FFA61901E006F8010B15F8010B8742F9D115F8014B002CE9D115F8010B2C7805
:20FA780000022418D4D1BDE8F08142F24011C4F208010B684A6D410838BF012108D303F0D7
:20FA9800010102F004020A434FF0000118BF0121820805D3002211B1990828BF0122114686
:20FAB800C00805D3002011B1D90828BF01200146002914BF0120022070470000F8B506468D
:20FAD8000F4D104F7388002417E0A00000EBC400321851689068D26852B9AF420BD00A7860
:20FAF80055F822200346491C08461946904701E0FFF78DFE7388641CA4B2A342E5DCF8BD9F
:20FB180028FE010034FE010000BF704708B5FFF7FBFFFEE738B50546094800688047094C5E
:20FB3800201D006810B1014628468847206800B18047054800688047FFF7E8FF38BDC0466F
:20FB580008010020100100200C0100200B4885460B4885446F4607208743BD4609486F461D
:20FB7800076000F0DFF8002801D0FFF713FF00F0A5F80120FFF7CEFFFEE7C046FC2B00209B
:20FB980000010000180100204FF6405110B5C0F2010151F8201046F2000241F2000442F2A6
:20FBB800D003C2F20002C4F20804C4F2020362501968012202FA00F08143196010BD4FF696
:20FBD800405110B5C0F2010151F8201041F2000442F2D0024FF4C043C4F20804C4F202028B
:20FBF80063501368012101FA00F01843106010BD08B5FFF732FA002008BD704708B5FFF7EC
:20FC180048FB08B1002001E04FF0FF3008BD08B5FFF76DFB08B1002001E04FF0FF3008BD94
:20FC38004FF6C052810910B5C0F2010201F03C01525842F20003C4F208039C5800F00F008E
:20FC5800012101FA00F02043985010BD08B540F2A813C1F200031B689B69984740F28442A9
:20FC78000021C4F26022116008BD40F2A81108B5C1F2000109684969884740F28442002176
:20FC9800C4F26022116008BD4FF64053C0F2010353F82000114341F20003C4F20803195031
:20FCB80070474368002923F00C0318BF43F00803002A18BF43F00403436070470449B1F1E6
:20FCD800FF3F07BF0020011C0868091DFFF795BCFFFFFFFF0349086070470249091F0860AC
:20FCF800704770470C010020426801F0030122F00302114341607047D0F80320C31D0846D6
:20FD18001946FFF784BDEFF3108062B6704700207047D0F8032008460021FFF7CABD012223
:08FD3800FFF76EBE01207047C9
:20FD40000000000004000000080000000C0000001000000014000000180000001C00000033
:20FD60002000000024000000280000002C0000003000000034000000380000003C00000013
:20FD80004000000044000000480000004C0000005000000054000000580000005C000000F3
:20FDA0006000000064000000680000006C0000007000000074000000780000007C000000D3
:20FDC00054000000780000006C000000600000003C0000004800000084000000580000002B
:20FDE0007C0000007000000064000000400000004C000000880000005C00000080000000C3
:14FE0000740000006800000044000000500000008C000000F2
:20FE18000002FBFC0100FBFC01020D000200000037FD010011FD01002BFD0100000000005A
:18FE3800020000000801000018FE01000801002038FE01000000002010
:20FF300042494D205370656369616C202D3137204D617220313620323031362032333A32A2
:05FF5000303A353900D4
:20FF6000FFFFFFFFFFFFFFFFFFFFFFFFFFFFFFFFFFFFFFFFFFFFFFFFFFFFFFFFFFFFFFFFA1
:20FF8000FFFFFFFFFFFFFFFFFFFFFFFFFFFFFFFFFFFFFFFFFFFFFFFFFFFFFFFFFFFFFFFF81
:04FFA000FFFFFFFF61
:20FFA80000008001100082FFFDFF58003AEFBDF3FFFFFFFFFFFFFFFFFFFFFFFFFFFFFFFF0A
:20FFC800FFFFFFFFFFFFFFFFFFFFFFFFFFFFFFFFFFFFFFC5FFFFFFFFC5FFFFFFC5C5C5FF5B
:18FFE800C5C5C5FF00000000FFFFFFFFFFFFFFFFFFFFFFFFFFFFFFFFC3
:00000001FF
